BL51 BANKED LINKER/LOCATER V6.05                                                        09/02/2010  14:40:04  PAGE 1


BL51 BANKED LINKER/LOCATER V6.05, INVOKED BY:
C:\KEIL\C51\BIN\BL51.EXE STARTUP.obj, EKTC52C .obj TO EKTC52-ENG RAMSIZE (256) CODE (0X0000-0X3FFF)


MEMORY MODEL: COMPACT


INPUT MODULES INCLUDED:
  STARTUP.obj (?C_STARTUP)
  EKTC52C .obj (EKTC52C_)
  C:\KEIL\C51\LIB\C51C.LIB (?C_INIT)
  C:\KEIL\C51\LIB\C51C.LIB (?C?CLDPTR)


LINK MAP OF MODULE:  EKTC52-ENG (?C_STARTUP)


            TYPE    BASE      LENGTH    RELOCATION   SEGMENT NAME
            -----------------------------------------------------

            * * * * * * *   D A T A   M E M O R Y   * * * * * * *
            REG     0000H     0008H     ABSOLUTE     "REG BANK 0"
            REG     0008H     0008H     ABSOLUTE     "REG BANK 1"
            IDATA   0010H     0001H     UNIT         ?STACK

            * * * * * * *  X D A T A   M E M O R Y  * * * * * * *
            XDATA   0000H     00A4H     INPAGE       ?PD?EKTC52C_

            * * * * * * *   C O D E   M E M O R Y   * * * * * * *
            CODE    0000H     0003H     ABSOLUTE     
                    0003H     0008H                  *** GAP ***
            CODE    000BH     0003H     ABSOLUTE     
            CODE    000EH     000EH     UNIT         ?PR?_UART0_TRANSMIT?EKTC52C_
                    001CH     0007H                  *** GAP ***
            CODE    0023H     0003H     ABSOLUTE     
            CODE    0026H     008EH     UNIT         ?PR?UART0_ISR?EKTC52C_
            CODE    00B4H     008CH     UNIT         ?C_C51STARTUP
            CODE    0140H     0065H     UNIT         ?PR?MAIN?EKTC52C_
            CODE    01A5H     002AH     UNIT         ?PR?SYSINIT?EKTC52C_
            CODE    01CFH     0029H     UNIT         ?C_INITSEG
            CODE    01F8H     0023H     UNIT         ?PR?TIMER0?EKTC52C_
            CODE    021BH     0021H     UNIT         ?PR?_SEND_STR?EKTC52C_
            CODE    023CH     0019H     UNIT         ?C?LIB_CODE
            CODE    0255H     000BH     UNIT         ?PR?EN?EKTC52C_
            CODE    0260H     000AH     UNIT         ?PR?_DELAY_MS?EKTC52C_
            CODE    026AH     000AH     UNIT         ?PR?_PIC_STR?EKTC52C_



OVERLAY MAP OF MODULE:   EKTC52-ENG (?C_STARTUP)


SEGMENT
  +--> CALLED SEGMENT
---------------------
?C_C51STARTUP
  +--> ?PR?MAIN?EKTC52C_
  +--> ?C_INITSEG
BL51 BANKED LINKER/LOCATER V6.05                                                      09/02/2010  14:40:04  PAGE 2



?PR?MAIN?EKTC52C_
  +--> ?PR?SYSINIT?EKTC52C_
  +--> ?PR?_DELAY_MS?EKTC52C_
  +--> ?PR?_SEND_STR?EKTC52C_
  +--> ?PR?EN?EKTC52C_
  +--> ?PR?_PIC_STR?EKTC52C_

?PR?_SEND_STR?EKTC52C_
  +--> ?PR?_UART0_TRANSMIT?EKTC52C_

?PR?EN?EKTC52C_
  +--> ?PR?_SEND_STR?EKTC52C_

?PR?_PIC_STR?EKTC52C_
  +--> ?PR?_SEND_STR?EKTC52C_
  +--> ?PR?EN?EKTC52C_



SYMBOL TABLE OF MODULE:  EKTC52-ENG (?C_STARTUP)

  VALUE           TYPE          NAME
  ----------------------------------

  -------         MODULE        ?C_STARTUP
  C:00B4H         SEGMENT       ?C_C51STARTUP
  I:0010H         SEGMENT       ?STACK
  C:0000H         PUBLIC        ?C_STARTUP
  D:00E0H         SYMBOL        ACC
  D:00F0H         SYMBOL        B
  D:0083H         SYMBOL        DPH
  D:0082H         SYMBOL        DPL
  N:0000H         SYMBOL        IBPSTACK
  N:0100H         SYMBOL        IBPSTACKTOP
  N:0080H         SYMBOL        IDATALEN
  C:00B7H         SYMBOL        IDATALOOP
  N:0000H         SYMBOL        PBPSTACK
  N:0100H         SYMBOL        PBPSTACKTOP
  N:0000H         SYMBOL        PDATALEN
  N:0000H         SYMBOL        PDATASTART
  N:0000H         SYMBOL        PPAGE
  N:0000H         SYMBOL        PPAGEENABLE
  D:00A0H         SYMBOL        PPAGE_SFR
  D:0081H         SYMBOL        SP
  C:00B4H         SYMBOL        STARTUP1
  N:0000H         SYMBOL        XBPSTACK
  N:0000H         SYMBOL        XBPSTACKTOP
  N:0000H         SYMBOL        XDATALEN
  N:0000H         SYMBOL        XDATASTART
  C:0000H         LINE#         126
  C:00B4H         LINE#         133
  C:00B6H         LINE#         134
  C:00B7H         LINE#         135
  C:00B8H         LINE#         136
  C:00BAH         LINE#         185
  C:00BDH         LINE#         196
BL51 BANKED LINKER/LOCATER V6.05                                                      09/02/2010  14:40:04  PAGE 3


  -------         ENDMOD        ?C_STARTUP

  -------         MODULE        EKTC52C_
  C:0000H         SYMBOL        _ICE_DUMMY_
  D:0090H         PUBLIC        P1
  D:00B0H         PUBLIC        P3
  B:00A8H.7       PUBLIC        EA
  D:00A8H         PUBLIC        IE
  B:00A8H.4       PUBLIC        ES
  D:00B8H         PUBLIC        IP
  B:0098H.0       PUBLIC        RI
  B:0098H.1       PUBLIC        TI
  X:0000H         PUBLIC        color
  C:0140H         PUBLIC        main
  C:000EH         PUBLIC        _Uart0_transmit
  X:0006H         PUBLIC        Tim
  D:0099H         PUBLIC        SBUF
  D:0087H         PUBLIC        PCON
  C:01F8H         PUBLIC        Timer0
  D:0098H         PUBLIC        SCON
  D:0089H         PUBLIC        TMOD
  D:0088H         PUBLIC        TCON
  X:0007H         PUBLIC        end
  X:000BH         PUBLIC        rec_flag
  X:000CH         PUBLIC        rec
  C:0026H         PUBLIC        UART0_ISR
  X:008CH         PUBLIC        pic
  X:008FH         PUBLIC        clr
  B:00A8H.1       PUBLIC        ET0
  B:0088H.5       PUBLIC        TF0
  D:008CH         PUBLIC        TH0
  D:008DH         PUBLIC        TH1
  D:008AH         PUBLIC        TL0
  D:008BH         PUBLIC        TL1
  C:0255H         PUBLIC        en
  C:0260H         PUBLIC        _delay_ms
  B:0088H.4       PUBLIC        TR0
  C:01A5H         PUBLIC        SysInit
  B:0088H.6       PUBLIC        TR1
  X:0091H         PUBLIC        LEN
  C:0223H         PUBLIC        _send_str
  D:00C8H         PUBLIC        T2CON
  X:0092H         PUBLIC        i
  X:0093H         PUBLIC        j
  X:0095H         PUBLIC        clr1
  C:026AH         PUBLIC        _pic_str
  D:00D0H         PUBLIC        PSW
  -------         PROC          TIMER0
  C:01F8H         LINE#         63
  C:01FFH         LINE#         65
  C:0201H         LINE#         66
  C:0203H         LINE#         67
  C:0206H         LINE#         68
  C:0209H         LINE#         71
  C:0214H         LINE#         106
  C:0216H         LINE#         107
  -------         ENDPROC       TIMER0
BL51 BANKED LINKER/LOCATER V6.05                                                      09/02/2010  14:40:04  PAGE 4


  -------         PROC          UART0_ISR
  -------         DO            
  D:0007H         SYMBOL        temp
  -------         ENDDO         
  C:0026H         LINE#         113
  C:0035H         LINE#         116
  C:0038H         LINE#         117
  C:0038H         LINE#         118
  C:0045H         LINE#         119
  C:0054H         LINE#         120
  C:005BH         LINE#         122
  C:0080H         LINE#         123
  C:0080H         LINE#         124
  C:008DH         LINE#         125
  C:0098H         LINE#         126
  C:00A1H         LINE#         127
  C:00A1H         LINE#         129
  C:00A3H         LINE#         130
  C:00A5H         LINE#         132
  C:00A5H         LINE#         133
  C:00A7H         LINE#         134
  C:00A7H         LINE#         135
  -------         ENDPROC       UART0_ISR
  -------         PROC          _UART0_TRANSMIT
  D:0007H         SYMBOL        i
  C:000EH         LINE#         140
  C:000EH         LINE#         141
  C:000EH         LINE#         142
  C:0010H         LINE#         143
  C:0012H         LINE#         144
  C:0014H         LINE#         145
  C:0017H         LINE#         146
  C:0019H         LINE#         147
  C:001BH         LINE#         148
  -------         ENDPROC       _UART0_TRANSMIT
  -------         PROC          L?0040
  -------         ENDPROC       L?0040
  -------         PROC          _SEND_STR
  D:0001H         SYMBOL        p
  D:0005H         SYMBOL        s
  -------         DO            
  D:0006H         SYMBOL        m
  -------         ENDDO         
  C:0223H         LINE#         150
  C:0223H         LINE#         151
  C:0223H         LINE#         153
  C:022AH         LINE#         154
  C:022AH         LINE#         155
  C:0231H         LINE#         156
  C:0238H         LINE#         157
  C:023BH         LINE#         158
  -------         ENDPROC       _SEND_STR
  -------         PROC          _DELAY_MS
  D:0007H         SYMBOL        n
  C:0260H         LINE#         163
  C:0260H         LINE#         164
  C:0260H         LINE#         165
BL51 BANKED LINKER/LOCATER V6.05                                                      09/02/2010  14:40:04  PAGE 5


  C:0264H         LINE#         166
  C:0269H         LINE#         167
  -------         ENDPROC       _DELAY_MS
  -------         PROC          SYSINIT
  C:01A5H         LINE#         172
  C:01A5H         LINE#         173
  C:01A5H         LINE#         188
  C:01A9H         LINE#         189
  C:01ACH         LINE#         190
  C:01B1H         LINE#         192
  C:01B4H         LINE#         193
  C:01B7H         LINE#         194
  C:01BAH         LINE#         195
  C:01BDH         LINE#         196
  C:01C0H         LINE#         197
  C:01C2H         LINE#         198
  C:01C4H         LINE#         199
  C:01C7H         LINE#         200
  C:01CAH         LINE#         201
  C:01CCH         LINE#         202
  C:01CEH         LINE#         203
  -------         ENDPROC       SYSINIT
  -------         PROC          EN
  C:0255H         LINE#         208
  C:0255H         LINE#         209
  C:0255H         LINE#         210
  -------         ENDPROC       EN
  -------         PROC          _PIC_STR
  D:0007H         SYMBOL        i
  C:026AH         LINE#         216
  C:026AH         LINE#         217
  C:026AH         LINE#         218
  C:026EH         LINE#         219
  C:0271H         LINE#         220
  -------         ENDPROC       _PIC_STR
  -------         PROC          MAIN
  C:0140H         LINE#         279
  C:0140H         LINE#         280
  C:0140H         LINE#         281
  C:0142H         LINE#         282
  C:0145H         LINE#         283
  C:0147H         LINE#         285
  C:014CH         LINE#         286
  C:0150H         LINE#         287
  C:015BH         LINE#         288
  C:015EH         LINE#         289
  C:0163H         LINE#         290
  C:0168H         LINE#         291
  C:016DH         LINE#         293
  C:016DH         LINE#         294
  C:016DH         LINE#         295
  C:0175H         LINE#         296
  C:0175H         LINE#         297
  C:017BH         LINE#         298
  C:017BH         LINE#         300
  C:017BH         LINE#         301
  C:0180H         LINE#         302
BL51 BANKED LINKER/LOCATER V6.05                                                      09/02/2010  14:40:04  PAGE 6


  C:0180H         LINE#         304
  C:0180H         LINE#         305
  C:0184H         LINE#         306
  C:0184H         LINE#         307
  C:0189H         LINE#         308
  C:018EH         LINE#         309
  C:0197H         LINE#         310
  C:019AH         LINE#         311
  C:019DH         LINE#         312
  C:019DH         LINE#         313
  C:019FH         LINE#         321
  C:01A3H         LINE#         322
  C:01A3H         LINE#         324
  C:01A3H         LINE#         407
  -------         ENDPROC       MAIN
  -------         ENDMOD        EKTC52C_

  -------         MODULE        ?C?CLDPTR
  C:023CH         PUBLIC        ?C?CLDPTR
  -------         ENDMOD        ?C?CLDPTR

Program Size: data=17.0 xdata=164 code=613
LINK/LOCATE RUN COMPLETE.  0 WARNING(S),  0 ERROR(S)
